:020000040000FA
:02000000812855
:020008005E2A6E
:10001000D10000300D28D1004030D20048207C3083
:10002000512052085120510851204D20182008001D
:100030000A30CC001B28CC0B1A28080028304A2292
:10004000383008203930082014300820703008205B
:10005000563008206C300820C8304A22383008203A
:100060000C3008200130082001304A223D220800CF
:1000700044208A110A12D00A0319CF0A003E03193C
:1000800043280B20382808004F088A0050088200B7
:100090008514051405108510080085140510051435
:1000A0000800D3000830D4000510D31B05148514B4
:1000B0008510D30DD40B5428831605148312851490
:1000C0000000851083160510831208000830D40044
:1000D0008316051483128514031005180314D30D19
:1000E0008510D40B6B288316051083125308080063
:1000F0000510851485100514080005148514851055
:10010000080083018B0185010730990083163C307C
:10011000850034309700950070308F0008308100E2
:10012000831281018B128B170514851447221E2020
:100130000C3008200230CB00803008200030CF0087
:10014000BD30D0003820C030082038205822582236
:10015000803008203820C03008203820582258220B
:10016000CB0B9C280130082058225822EA206F210E
:10017000C60146150530C500152946346D34533483
:1001800074346534723465346F3400342034203470
:1001900052346134643469346F342034003456345A
:1001A00065347234203431342E34303434340034F5
:1001B00020346234793420344D342E345934203490
:1001C0000034203456346F346C343D3420342034C1
:1001D00020340034831626309B0083124330840081
:1001E0000230CB0083161C141A089B0A831280006D
:1001F000840ACB0BF2280800831626309B0083125A
:10020000433084000230CB00000883169A001C158E
:1002100055309D00AA309D009C149C180D299B0A06
:100220008312840ACB0B04290800851E3B21051E7E
:100230004821851D5521051D6121461C2C296F2152
:10024000461043228B120530C2003830810027301F
:10025000C0001030C1008B16461D36294908CF005A
:100260004A08D0004611C03008203820C61C152985
:10027000FC20C61015294322851A45294614C303BC
:10028000430A031D45294508C300851E452908006A
:100290004322051A52294614C30A4308450203188B
:1002A0005229C301051E52290800432285195E29DF
:1002B0004614C403440A031D5E29C401851D5E293A
:1002C0000800432205196C294614C40A44080F3C4F
:1002D00003186C290F30C400051D6C29080001307B
:1002E000CF00AF30D0004308C9000310C90DC90DBD
:1002F0004908CA00C90D490D0318CF0A4A07031857
:10030000CF0AD0070318CF0A8030082038204F08C2
:10031000C9005008CA000930D0070318CF0A44208A
:10032000C700D00A0319CF0A4420C800C0300820F3
:100330000030CF00E130D00038200A3044020318EA
:10034000A529C63008204408AB29C5300820313023
:100350000B200A30440230380B20272208004D348D
:10036000493444342D3446344D3420342034003460
:100370002034373436342E3431344D3448347A34E2
:100380000034003458345A34493450342D3446340F
:100390004D342034203400342034373437342E3474
:1003A00038344D3448347A34003404349834463484
:1003B0004D342034413449344334483449340034D2
:1003C0002034383430342E3437344D3448347A3491
:1003D00000340B34D8344E3448344B342034463453
:1003E0004D342034203400342034383432342E3428
:1003F00035344D3448347A3400341034583454345D
:100400004F344B34413449342034203420340034C8
:100410002034393432342E3439344D3448347A343B
:1004200000342A34583443344234433420342034A2
:1004300020342034203400342034393433342E3402
:1004400037344D3448347A3400342C34583448200E
:1004500020305120D0305120013051204708512008
:100460004808512000305120003051208830512060
:100470004408803851204D2008002730CC00402A05
:10048000CC0B3F2A08001E304A2A64304A2AC83062
:100490004A2A0130CD00DD30CC004E2A4F2A502AA6
:1004A000CC0B4D2A0000542A552ACD0B4B2A0800AC
:1004B0000A30CE004522CE0B5A2A0800F00003086D
:1004C000F10083120B1D7E2A0B11383081000130A0
:1004D000C10203196F2A03187E2AC0027E2AC008AF
:1004E000031D7E2A2730C0001030C10005304202B3
:1004F00003194615C20B7E2AC6148B12710883009D
:06050000F00E700E090070
:02400E00C43FAD
:1042000043006F0070007900720069006700680069
:1042100074002000280043002900200032003000F4
:10422000320030002D00320030003200310020001A
:104230006200790020004D002E00590061006D00E1
:1042400061006D006F0074006F00FF00030001004B
:00000001FF
